:020000040000FA
:020000007B285B
:080008000000F800030E830163
:10001000F9000A08FA008A010408FB00831203139E
:10002000101083120313BE308E00EE308F00831247
:100030000313FC03031D1F28FD0AC830FC00043015
:10004000A006201D2B2823080F398A110A12002729
:10005000803887003128230E0F398A110A120027B1
:100060008700831203130C10831603130C148312DE
:1000700003131014831203137B0884007A088A0088
:10008000790E8300F80E780E0900831203130B1704
:100090008B1783120313003083120313C830FC0044
:1000A000831203130C10831603130C14831203130F
:1000B000101483120313FD01A101A2010030A50059
:1000C0003C30A40008008312031385018601FF3031
:1000D0008700831203179E01831203179F01831663
:1000E00003130B308500FF3086008701C0308B0082
:1000F000831203130800A00163204520A201A3017D
:10010000A80120178D206C219820A018B220C120B2
:10011000E32006213621B5208228A01D9528AC0AAF
:100120002208AC1FFF30A30008002208A30008002B
:10013000201C08007D08210203190800A10AA4035D
:10014000031D0800A5080319A728A5030800A0148B
:100150000030A5003C30A4000800A010FC017D0880
:10016000A100A828A0103E210800201CBC28A01B2C
:1001700008000515A0170800A01F08000511A0130E
:100180000800A901A701061BC7282914A70A851979
:10019000CB28A914A70A861ACF282915A70A061A58
:1001A000D328A915A70A8518D7282916A70A05183C
:1001B000DB28A916A70AA908031908002708013C8B
:1001C000031DA9170800A908031DE8282016080028
:1001D000201EF328AA01AB012012A91B0800290840
:1001E000A800A0120800AA0A0319AB0A2A08003CBA
:1001F000031D08002B08023C031D08002908A80065
:10020000A016C030AA000130AB000800280803196E
:100210000800A01128191821A8191B21281A1E212D
:10022000A81A212128182421A8183021A801080083
:10023000201C20174D29201C20173E29201C201788
:100240006529201C20175E2920180800A208031920
:1002500008002014201BAD207D08A10020130800F9
:100260002010A01E0800A20120170800201C080072
:10027000A208031D08002017A01530292208031921
:1002800008000F3903194629A2030800A20E220311
:100290000F399038A200A20E08002208993C0319D9
:1002A000080022080F39093C03195829A20A08003E
:1002B000A20E220A0F39A200A20E08000A30A700DF
:1002C0003E21A703031D602908000A30A7004D2125
:1002D000A703031D67290800A701A703031D6D29B4
:0202E000080014
:100E0000A60007308A00260882074034793424344B
:100E10003034193412340234783400341034083445
:0A0E200003344634213406347F34D5
:02400E00D130AF
:00000001FF
